:03000000020606EF
:0C060600787FE4F6D8FD75812102064DD6
:100422000D0A3D3D3D20493243E689ABE68F8FE719
:10043200BB93E69E9C203D3D3D0D0A00E5BA94E744
:10044200AD94E59CB0E59D80E58897E8A1A8EFBC56
:100452008837E4BD8DEFBC893A0D0A00307825302B
:10046200325820000D0A00E5AFB9E5BA94E58F9144
:10047200E98081E59CB0E59D80EFBC8838E4BD8DC4
:10048200E58699E6A8A1E5BC8FEFBC893A0D0A0082
:10049200E69CAAE6A380E6B58BE588B0E4BBBBE4A4
:1004A200BD95493243E8AEBEE5A4870D0A003D3D45
:1004B2003D3D3D3D3D3D3D3D3D3D3D3D3D3D3D3D6A
:1004C2000D0A003D3D3D3D3D3D3D3D3D3D3D3D3DFA
:1004D2003D3D3D3D3D3D3D3D3D3D3D3D3D3D3D3D4A
:1004E2003D3D3D3D3D3D3D3D3D3D3D0D0A00202014
:1004F2005354433847314B303820493243E8AEBE7B
:10050200E5A487E689ABE68F8FE599A80D0A00E797
:10051200B3BBE7BB9FE5889DE5A78BE58C96E5AE6F
:100522008CE688902E2E2E0D0A00E6AF8F35E7A7B7
:1005320092E887AAE58AA8E689ABE68F8FE4B880BD
:10054200E6ACA1493243E680BBE7BABF0D0A000D13
:100552000A5BE5BC80E5A78BE689ABE68F8F2E2E82
:100562002E5D0D0A005BE689ABE68F8FE5AE8CE669
:0605720088905D0D0A00F7
:03081500011D00C2
:0300C300020755DC
:10075500C0E0C083C082C0BA43BA8090FE82E03058
:10076500E606E054BFF0C209D0BAD082D083D0E00B
:010775003251
:10077600E4FDFCC3ED9FEC9E5015E4FBFA0BBB00B9
:0F078600010ABA04F8BB4CF50DBD00010C80E46C
:010795002241
:0F07D30090FE82E030E6F990FE82E054BFF02203
:0C07F100D20990FE817481F02009FD22E5
:1007C20090FE86EFF0D20990FE817482F02009FD3E
:0107D2002204
:0C07FD00D20990FE817483F02009FD22D7
:0C080900D20990FE817486F02009FD22C7
:10079600759204E4F59175BA8090FE8074F3F0903A
:0707A600FE82E4F0D2AF2255
:10073200C200EF7002C3221207F1EF25E0FF120799
:10074200C21207FD90FE82E020E102D200120809E7
:02075200A20003
:010754002282
:10070400E4F51DF9AF01120732501EE51DC39480B4
:100714005010AF1D051D74002FF582E43400F583DD
:0D072400E9F07F017E0012077609B980D749
:0107310022A5
:1007AD00759850438E01538EFB75D7FE75D6FF435A
:0507BD008E10D299220C
:0800B8008F993099FDC29922D5
:100003007BFF7A047922120128E51DD39400500363
:100013000200A67BFF7A04793E120128E4F508E585
:1000230008C3951D502B7BFF7A04795E7400250865
:10003300F582E43400F583E0F50C120128E50804A9
:10004300540770097BFF7A0479661201280508803A
:10005300CE7BFF7A0479661201287BFF7A047969E3
:10006300120128E4F508E508C3951D502E7BFF7A9D
:1000730004795E74002508F582E43400F583E0FF1B
:1000830025E0F50C120128E50804540770097BFFED
:100093007A047966120128050880CB7BFF7A0479FC
:1000A3006680067BFF7A0479921201287BFF7A042B
:0500B30079B0020128F4
:0E07E20000007FD37E1E7D0BDDFEDEFCDFFA05
:0107F00022E6
:100692001207961207ADC2927BFF7A0479661201A5
:1006A200287BFF7A0479C51201287BFF7A0479F04E
:1006B2001201287BFF7A0479C51201287BFF7A0593
:1006C20079111201287BFF7A05792C1201287BFF10
:1006D2007A0479C5120128D2927F647E00120776CD
:1006E200C2927BFF7A0579511201281207047BFF1F
:1006F2007A057967120128120003E4F51D1207E258
:0207020080D5A0
:10061200020692E493A3F8E493A34003F68001F266
:1006220008DFF48029E493A3F85407240CC8C333E9
:10063200C4540F4420C8834004F456800146F6DFB8
:10064200E4800B0102040810204080900815E47E2B
:10065200019360BCA3FF543F30E509541FFEE493AD
:10066200A360010ECF54C025E060A840B8E493A374
:10067200FAE493A3F8E493A3C8C582C8CAC583CA9F
:10068200F0A3C8C582C8CAC583CADFE9DEE780BE57
:0108180000DF
:1000C600E518240CF8E60518227809300702780CA2
:1000D600E475F0011205D00205782000EB7F2ED2E0
:1000E600008018EF540F2490D43440D4FF30040B12
:1000F600EF24BFB41A0050032461FFE5196002150E
:1001060019051CE51C7002051B30070D7809E475FE
:10011600F0011205D0EF0205BE0200B87403D20743
:100126008003E4C207F5188B098A0A890BE4F519DE
:10013600F51BF51CE51960077F2012010180F57596
:100146001AFFC201C200C202C203C205C206C20829
:100156001200CFFF700D3007057F00120112AF1C91
:10016600AE1B22B4255FC2D5C2041200CFFF24D035
:10017600B40A00501A75F00A781930D50508B6FF8A
:100186000106C6A426F620D5047002D20380D9241F
:10019600CFB41A00EF5004C2E5D204020312D20112
:1001A60080C6D20080C0D20280BCD2D580BAD20529
:1001B60080B47F201201012002077401B5190040A6
:1001C600F11200C6FF12010102013AD208D20680DE
:1001D600951200C6FB1200C6FA1200C6F94A4B7009
:1001E6000679E37A037BFF20022EE519602A7E005A
:1001F6008E8275830012059160060EEE651A70F008
:10020600C2D5EBC0E0EAC0E0E9C0E0EE120359D087
:10021600E0F9D0E0FAD0E0FB120578FF60AAEBC067
:10022600E0EAC0E0E9C0E0120101D0E02401F9D023
:10023600E03400FAD0E0FBE51A0460DCD51AD98078
:10024600877BFF7A037955D202809C7910800279E8
:1002560008C206C2088008D2D5790A8004790AC283
:10026600D5E51A047002F51AE4FAFDFEFF1200C67F
:10027600FC7B082001131200C6FD7B1030000A1219
:1002860000C6FE1200C6FF7B20EC3382D592D55005
:1002960013C3E43000069FFFE49EFEE42001039DA5
:1002A600FDE49CFCE4CBF8C201EC700CCFCECDCCC7
:1002B600E824F8F870F38017C3EF33FFEE33FEED52
:1002C60033FDEC33FCEB33FB994002FB0FD8E9EB33
:1002D600300105F8D0E0C448B201C0E00AEC4D4E4A
:1002E6004F78207B0070C2EAB51A0040BCC0E0120D
:1002F600035BD0F0D0E0200104C4C0E0C4B201C06A
:10030600F01200EAD0F0D5F0EB02013A1205E00156
:10031600D75302515801A84C01A44202554F025D21
:0F03260044025D4901BD43026355024746024749
:100335004502474704035001AC2D01B02E01D32BD4
:1003450001B42301D12003EC2A016C48000001CB44
:100355003F3F3F00790AA2D5200314300509B910A3
:10036500020404B9080104A2D520060250010420A4
:1003750002689202B519005034C0E07F203003199D
:100385007F30A20272067205500F1203B2C202C27A
:1003950006C205C2087F30800F300503E9C0E012B0
:1003A5000101300503D0E0F9D0E0B519CC300517CF
:1003B5007F30B9100C1201017F583004077F788017
:1003C50003B908031201013002057F2D0201017FE7
:1003D500202008F87F2B2006F322920280CF286E7A
:1003E500756C6C2900D2011200C63001F8C2017883
:1003F5001930D50108F602016C2D504349581200F9
:10040500C62403B405004001E49003FE931200F2F4
:0D041500743A1200F2D2037519040202516C
:10057800BB010689828A83E0225002E722BBFE0281
:09058800E32289828A83E49322B4
:10059100BB010CE58229F582E5833AF583E022501F
:1005A10006E92582F8E622BBFE06E92582F8E22269
:0D05B100E58229F582E5833AF583E4932283
:1005BE00BB010689828A83F0225002F722BBFE011C
:0205CE00F32216
:1005D000FAE6FB0808E6F925F0F618E6CA3AF6222C
:1005E000D083D082F8E4937012740193700DA3A3AA
:1005F00093F8740193F5828883E4737402936860BE
:06060000EFA3A3A380DFBD
:00000001FF
